:10000000FFC3FFC3FFC3FFC3FFC3FFC3FFC3FFC3E0
:10001000FFC3FFC3FFC3FFC3FFC3FFC3FFC3FFC3D0
:10002000FFC3FFC3FFC3FFFFFFFFFFFFFFFFFFFF94
:10003000FFFFFFFFFFFFFFFFFFFFFFFFFFFFFFFFD0
:10004000FFFFFFFFFFFFFFFFFFFFFFFFFFFFFFFFC0
:10005000FFFFFFFFFFFFFFFFFFFFFFFFFFFFFFFFB0
:10006000FFFFFFFFFFFFFFFFFFFFFFFFFFFFFFFFA0
:1008000055C0D8C46EC06DC06CC06BC06AC069C032
:1008100068C067C066C065C064C063C062C061C0B4
:1008200060C05FC05EC072C171C173C172C171C16D
:1008300073C172C174C173C175C177C1090212005D
:1008400001010080320904000000000000001201D4
:100850001001FF000008C016DC05000101020001C4
:100860001C03450045002D00500072006F0067001A
:100870002000760031002E00300030002C03730081
:100880003200300030003000730061006D006900FC
:1008900072006800400067006D00610069006C0034
:1008A0002E0063006F006D000403090411241FBEB5
:1008B000CFE5D4E0DEBFCDBF10E0A0E6B0E0ECE6CF
:1008C000F4E102C005900D92A038B107D9F711E00C
:1008D000A0E8B0E001C01D92A03CB107E1F77ED5D1
:1008E000C3C58ECF1F93CF93DF93182FD92FC62F59
:1008F0008091810090918200009729F0A12FBD2F57
:1009000020E030E02BC0959A6091850070918600C0
:100910000090890002C0660F771F0A94E2F780E01A
:1009200090E040918700509188002CE830E01AD187
:1009300090938B0080938A00959820918700309146
:10094000880082179307B9F4D9CFF901E457FF4F14
:10095000E80FF91F80818D932F5F3F4F80918100B9
:10096000909182002C1788F38C0F911D9093820038
:100970008093810001C0CFEF8C2FDF91CF911F9129
:1009800008952091810030918200DC0180E090E0A8
:1009900008C04D91F901E457FF4FE80FF91F40835C
:1009A00001968617B0F34091810050918200460F66
:1009B000511D509382004093810080918700909157
:1009C000880048175907F9F4959A6091850070914D
:1009D00086000090890002C0660F771F0A94E2F734
:1009E00080E090E02CE830E054D290938B0080932C
:1009F0008A0095982091870030918800821793078C
:100A000021F481E0089580E008958FEF0895CF9359
:100A1000DF93EC01888180768034A1F58981813073
:100A200011F0823011F510928200109281008A81BB
:100A300061D0909388008093870037D0809389009D
:100A40008B8128D03D8120E08C8190E0822B932BFC
:100A500090938600809385008A8175D0909384005E
:100A6000809383008FEF9FEF0FC0833059F4959AE6
:100A700080E690E090939F0180939E01959881E09D
:100A800090E002C080E090E0DF91CF91089588E48B
:100A900080B90895813011F488E405C0823011F4E2
:100AA0008CE001C081E080B9089580918E01909121
:100AB0008F0180329105A1F08132910538F48830A0
:100AC000910561F08031910589F412C0803891055B
:100AD00049F021E08030920749F406C083E0089590
:100AE00085E0089587E0089588E0089586E00895F8
:100AF00084E0089580938D0190E001978B309105FB
:100B0000D8F48D5E9B4F8F939F93089588E090E07B
:100B10000EC080E190E00BC080E290E008C080E46D
:100B200090E005C080E890E002C080E091E0909302
:100B30008F0180938E01089580E490E090938F015F
:100B400080938E01089581508B3048F4E82FF0E0B7
:100B5000EE0FFF1FE959FF4F80819181089580E0DA
:100B600092E00895CF93DF93DC01CB01FA01E90114
:100B700020918D012330D8F0263018F02B30B9F4B5
:100B80000AC0AC01BD0137E076956795579547954A
:100B90003A95D1F709C0AC01BD012FE07695679574
:100BA000579547952A95D1F74E75406A01C040EA9E
:100BB000592F39EC315009F495C024EA26BF06B606
:100BC00007FEFDCF21B1287F20938C01203129F031
:100BD000283399F3283009F085C043B924E826BFAB
:100BE00006B607FEFDCF21B1287F20938C0120326D
:100BF00009F3283311F3283109F065C020918D01E4
:100C0000263090F053B924E826BF06B607FEFDCF84
:100C100021B1287F20938C01203309F45EC0283352
:100C200061F2283209F04FC083B924E826BF06B626
:100C300007FEFDCF21B1287F20938C01203309F4DA
:100C40004CC0283309F4B9CF2832E9F524EA26BF8D
:100C500006B607FEFDCF21B1287F20938C012031FD
:100C600029F0283309F4A9CF283051F5242F216029
:100C700023B924E826BF06B607FEFDCF21B1287FA1
:100C800020938C01203411F1283439F12833C1F438
:100C900094CFE130F10509F434E836BF06B607FE1B
:100CA000FDCF21B1287F20938C01203521F02835FC
:100CB00039F4E0E0F0E023B129930196319709C0BF
:100CC00081E690E0A3D384E986BF0CC080E090E089
:100CD00034EC1E161F06ECF202C080E090E024E91E
:100CE00026BF02C08FEF9FEFDF91CF910895CF9283
:100CF000DF92FF920F931F93CF93DF93DC01CB0121
:100D00006A01D22FC32F20918D012330F0F02630BD
:100D100018F02B30D1F40AC0AC01BD01F7E0769594
:100D2000679557954795FA95D1F709C0AC01BD0174
:100D3000EFE07695679557954795EA95D1F75EE58B
:100D4000F52EF42220EAF22A02C040EAF42EE091C5
:100D50008E01F0918F0131978C019D01025010405E
:100D600020403040A601662757FD6095762F040F7E
:100D7000151F261F371FAF0160E070E0482B592B6D
:100D80006A2B7B2B041715072607370720F4F6017B
:100D9000E80FF91F03C0E82BF92B3196492F39ECE6
:100DA000315009F46CC024EA26BF06B607FEFDCF19
:100DB00021B1287F20938C01203129F0283399F329
:100DC000283009F05CC0F3B824E826BF06B607FE59
:100DD000FDCF21B1287F20938C01203209F32833E5
:100DE00011F3283109F046C020918D01263080F0A2
:100DF00043B924E826BF06B607FEFDCF21B1287F00
:100E000020938C012033B1F0283369F2283291F518
:100E100083B924E826BF06B607FEFDCF21B1287F9F
:100E200020938C01203331F0283309F4BCCF2832D1
:100E300009F503C080E090E01FC0AF01481B590BCB
:100E4000ED2FFC2F80E090E00EC0219123B924E823
:100E500026BF06B607FEFDCF21B1287F20938C0167
:100E6000283241F401969A01281B390B12161306F9
:100E700064F302C08FEF9FEF24E926BF02C08FEF1B
:100E80009FEFDF91CF911F910F91FF90DF90CF9057
:100E90000895AF92BF92CF92DF92EF92FF920F939D
:100EA0001F93CF93DF936B017C01EA01590100E0AE
:100EB00010E0C701B601AE01950119DF2FEF8F3F9A
:100EC000920799F0AC01662757FD6095762FC40E06
:100ED000D51EE61EF71EC81BD90BA80EB91E080F9B
:100EE000191F1C161D062CF302C00FEF1FEFC801BF
:100EF000DF91CF911F910F91FF90EF90DF90CF90F6
:100F0000BF90AF900895CF93DF936091A00163509D
:100F100067FDBCC020919D018CE090E0821B91098F
:100F2000EC01CC55DE4F20919C012D3209F09AC086
:100F3000683009F0A9C023EC209390012AE52093A2
:100F40007D00109280002881207641F0CE015FDD87
:100F50002FEF8F3F920709F471C079C03A81109248
:100F600099012981222339F410929A0129E931E06B
:100F700082E090E05EC0253019F43093A1014DC0AD
:100F8000263009F041C0FC01EA55FE4F2081895509
:100F90009E4FFC018081813019F48EE498E004C0FA
:100FA000823049F48CE398E090939F0180939E01F6
:100FB00082E190E025C0833009F5222349F488EAD4
:100FC00098E090939F0180939E0184E090E018C088
:100FD000213049F48CE798E090939F0180939E0123
:100FE0008CE290E00DC0223049F480E698E09093C6
:100FF0009F0180939E018CE190E002C080E090E030
:1010000020E42093800023C0283061F0293019F4B7
:101010003093A30102C02A3041F029E931E080E099
:1010200090E007C023EA31E002C029E931E081E025
:1010300090E030939F0120939E0109C0288127FFF3
:1010400002C08E819F8120E82093800006C02E81FF
:101050003F812817390708F4C90190937F008093D6
:101060007E0012C08091800087FF0EC0CE0189DC17
:101070008F3F21F48EE180937D0006C0882321F00C
:1010800010927F0010927E001092A00180917D004E
:1010900084FF63C080917E0090917F00FFEF8F3FBF
:1010A0009F0709F45AC0BC018930910510F068E02F
:1010B00070E0861B970B90937F0080937E00809159
:1010C000900198E8892780939001C62F662371F1DB
:1010D0009091800097FF05C081E991E003DCC82F63
:1010E00023C020919E0180919F0196FF0CC0E22FAA
:1010F000F82FA1E9B1E084918D9331968C2F820F66
:101100008E17C9F70DC0A22FB82F81E991E03D914C
:10111000FC013193CF01FD013C2F320F3A17B9F793
:10112000F0939F01E0939E01C93070F481E991E052
:101130006C2F3CD0CC5FCC3071F08FEF9FEF909351
:101140007F0080937E0007C08FEF9FEF90937F001A
:1011500080937E00CEE1C0937D0084E190B39474CF
:1011600031F48150D9F71092A10110929B01DF91C7
:10117000CF91089585B7826085BF8BB780648BBFA0
:101180000895A82FB92F80E090E041E050EA6095E3
:1011900030E009C02D9182279795879510F084271C
:1011A0009527305EC8F36F5FA8F30895EADF8D934B
:1011B0009D930895CF93CFB7CF93DF93C395869B2D
:1011C000E9F7869B0BC0869B09C0869B07C0869B60
:1011D00005C0869B03C0869B01C089C06F93C091E8
:1011E0009D01DD27CC55DE4F2F9365E5869B03C01F
:1011F0002F916F91E6CF0F931F934F9320E040E123
:101200005F9300B3047406FB27F93F9350E03BE083
:1012100039C0147440642F77012F5F5F1EC040688F
:1012200010B314742F7752501FC0406400B32F774F
:101230000474D1F15F5F00C023C0406210B32F7708
:10124000147491F15F5F00C025C0047410275150E1
:1012500012F45D5F0000115027952C3F10B3C8F6C3
:1012600014740127015027952C3FC8F64227499353
:1012700000B3047410274F73115027952C3FA8F624
:101280004695469510B3147479F0012701502795BF
:101290002C3F98F66B5A60F3315000B3B0F600C0A3
:1012A00010E41ABF002717C03B503195C31BD04034
:1012B00010E41ABF0881033CF9F00B34E9F02091E7
:1012C0009B011981110F1213EDCF093651F10D3227
:1012D00011F0013E39F70093A2013F915F914F91C8
:1012E0001F910F912F916F91CAB7C6FD67CFDF9104
:1012F000CF91CFBFCF9118952091A201222369F3FE
:101300001091A001112339F534303AF13093A00146
:1013100020939C0110919D013BE0311B30939D0176
:101320001CC00091A0010130B4F40AE530917D00A9
:1013300034FD14C000937D00C0E9D1E013C005273F
:1013400010E000C0000002BB1AC0052710E0221FF9
:101350001DC010E021C04AE502C032ED432FC4E1B8
:10136000D0E032E011B31464969A02B311BB54E496
:1013700020E865E320FF052702BB279517951C3F52
:10138000F0F66695B8F7B1F720FF052702BB279561
:1013900017951C3FD0F62795179517FF05270000D6
:1013A0001C3F02BBB0F629913A9519F70B7B1091BF
:1013B000A101110FC651D04002BB11F010939B0147
:1013C00010E41ABF006411B31B7B402F4B7B54E029
:1013D0005A95F1F702BB11BB42BB7FCF14BA80E331
:1013E00085BBC8DE54DB8D9AB89A9598C0988E9AC2
:1013F0008FEF99E6A8E181509040A040E1F700C04E
:1014000000008E98C09A78947EDDFECF0F931F93D4
:10141000CF93DF938C01E091BC01F091BD018381FA
:1014200081FF1AC0C0E0D0E005C00995009711F017
:10143000CFEFDFEFF80181918F016091BC017091D6
:10144000BD01DB011896ED91FC911997882369F78E
:101450008AE00995009711F0CFEFDFEFCE01DF9121
:10146000CF911F910F910895F894FFCF316572725B
:101470006F720010002000200040008000800000FB
:0C1480000100010002000200025AFFFF00
:00000001FF
